:100000000C94F9050C9440060C9440060C944006A0
:100010000C9440060C9440060C9440060C94400648
:100020000C9440060C9440060C94C60F0C944006A9
:100030000C94161E0C9440060C9440060C9440063A
:100040000C9440060C9440060C9440060C94400618
:100050000C9440060C94861E0C9440060C944006AA
:100060000C9440060C94E6090C9440060C9440064F
:100070000C9440060C9440060C9440060C944006E8
:100080000C9440060C9440060C9440060C944006D8
:100090000C9440060C9440060C9440060C944006C8
:1000A0000C9440060C9440060C9440066E07DE0744
:1000B000C007020816081C082008240828082C0875
:1000C0003008330837083B08BC10DE10CC11DE10B6
:1000D000CC1123114611CC119B11AE11B314B314E2
:1000E000E014E0143B1577156F176F178F156F1716
:1000F0008A168A1645176F176F175B178042803E66
:100100003C3A3B456843413F3D2B3567697A79006E
:1001100078141E806A801D16041A1F806B061B0748
:10012000082120806C2C1909171522806D11050BF0
:100130000A1C23806E80100D182425806F360E0C4B
:10014000122726807037380F33132D807175348055
:100150002F2E8072397D28308031807380648080BA
:1001600076802A778059745C5F66808062635A5D0E
:100170005E60295344575B565561478080808040BC
:10018000808080808080808080808080807E808071
:100190007C808080808080808080807B8001800364
:1001A0008080807F808080808080806580800280E9
:1001B000808080808080808080808080808080803F
:1001C000808080808080548080808080808080805B
:1001D0008080808080805880808080808080808047
:1001E00080808080804D80504A808080494C518042
:1001F0004F52808080804E80464B48800A002530D8
:100200003862003A200025303258000A722F6320ED
:1002100030313233343536370A00756E65787065A3
:1002200063746564207363616E20636F646520612D
:10023000742045305F46303A20253032580A007528
:100240006E6578706563746564207363616E2063A6
:100250006F64652061742046303A20253032580A98
:1002600000756E6578706563746564207363616E94
:1002700020636F64652061742046303A2046302840
:10028000636C65617220616E6420636F6E742E29E9
:100290000A00756E657870656374656420736361C8
:1002A0006E20636F64652061742045303A202530EC
:1002B00032580A00756E65787065637465642073E2
:1002C00063616E20636F646520617420494E4954F8
:1002D0003A20253032580A004F76657272756E0AE0
:1002E0000025690D0A00706275663A2066756C6CAF
:1002F0000A00505332205553415254206572726F98
:10030000723A202530325820646174613A202530D9
:1003100032580A004B6579626F61726420737461B0
:1003200072742E0A0055534220636F6E66696775BA
:100330007265642E0A000D0A696E69740A005B44D6
:100340005D005B435D003003500053002F0032001E
:1003500020006B006500790062006F006100720090
:100360006400200063006F006E007600650072007C
:1003700074006500720000000E0374002E006D0012
:100380002E006B002E0000000403090409028D00FA
:10039000050100A032090400000103010100092148
:1003A000110100012240000705810308000A090429
:1003B00001000103010200092111010001224D0089
:1003C0000705820308000A09040200010300000077
:1003D0000921110100012236000705830308000AE4
:1003E0000904030002030000000921110100012299
:1003F00022000705840320000107050403200001F3
:100400000904040001030000000921110100012278
:1004100039000705850320000112011001000000CA
:1004200008EDFE126501000102000105010906A1A7
:1004300001050719E029E7150025019508750181D7
:1004400002050819012905950575019102950175A7
:100450000391010507190029F71500250195F87585
:10046000018102C00631FF0974A10109751500263A
:10047000FF009520750881020976150026FF00957A
:100480002075089102C005010980A101850216812D
:100490000026B7001A81002AB70075109501810067
:1004A000C0050C0901A1018503160100269C021A52
:1004B00001002A9C02751095018100C00501090206
:1004C000A1010901A100050919012905150025014E
:1004D00095057501810295017503810105010930BA
:1004E00009311581257F9502750881060938158126
:1004F000257F950175088106050C0A3802158125AE
:100500007F950175088106C0C005010906A1010596
:100510000719E029E7150025019508750181029565
:1005200001750881010508190129059505750191D5
:10053000029501750391010507190029FF15002691
:10054000FF00950675088100C00A0025303258204A
:10055000006B6579626F6172645F7265706F72744F
:100560003A20004C45443A20253032580A00646550
:100570006C5F6B65795F6269743A2063616E2774A2
:100580002064656C3A20253032580A006164645F4B
:100590006B65795F6269743A2063616E27742061CC
:1005A00064643A20253032580A00290A0025750073
:1005B0002F002575005D28002564002000256400BB
:1005C000200025640020002564007C00253032587E
:1005D000006D6F7573656B6579205B62746E7C78F6
:1005E0002079207620685D287265702F61636C2900
:1005F0003A205B006D6B5F776865656C5F74696D51
:10060000655F746F5F6D6178203D2025640A006D21
:100610006B5F776865656C5F6D61785F737065654A
:1006200064203D2025640A006D6B5F74696D655F11
:10063000746F5F6D6178203D2025640A006D6B5FEB
:100640006D61785F7370656564203D2025640A00E4
:100650006D6B5F696E74657276616C203D202564F8
:100660000A006D6B5F64656C6179203D2025640A2A
:10067000006D6B5F776865656C5F74696D655F744D
:100680006F5F6D6178203D2025640A006D6B5F7798
:100690006865656C5F6D61785F7370656564203D4A
:1006A0002025640A006D6B5F74696D655F746F5F10
:1006B0006D6178203D2025640A006D6B5F6D617867
:1006C0005F7370656564203D2025640A006D6B5F73
:1006D000696E74657276616C203D2025640A006D38
:1006E0006B5F64656C6179203D2025640A000A0017
:1006F000257500363A20776865656C5F74696D65AD
:100700005F746F5F6D61783A20000A0025750035CF
:100710003A20776865656C5F6D61785F73706565B9
:10072000643A20000A00257500343A2074696D652A
:100730005F746F5F6D61783A20000A0025750033A1
:100740003A206D61785F73706565643A20000A0035
:10075000257500323A20696E74657276616C286D79
:1007600073293A20000A00257500313A2064656C2F
:100770006179282A31306D73293A20000A092D2029
:1007800056616C756573202D0A004D3E004D256441
:100790003E20003F007365742064656661756C746B
:1007A0000A00433E200077686572652064656C74BA
:1007B000613A20637572736F723D25642C207768EF
:1007C00065656C3D25640A53656520687474703AEC
:1007D0002F2F656E2E77696B6970656469612E6F66
:1007E00072672F77696B692F4D6F7573655F6B65E6
:1007F00079730A000A092D204D6F7573656B657951
:10080000202D0A4553432F713A09717569740A31D5
:100810003A0964656C6179282A31306D73290A328E
:100820003A09696E74657276616C286D73290A33B2
:100830003A096D61785F73706565640A343A0974CA
:10084000696D655F746F5F6D61780A353A09776825
:1008500065656C5F6D61785F73706565640A363AD3
:1008600009776865656C5F74696D655F746F5F6D4E
:1008700061780A0A703A097072696E742076616C48
:100880007565730A643A09736574206465666175F9
:100890006C74730A75703A092B310A646F776E3A7B
:1008A000092D310A706775703A092B31300A70676B
:1008B000646F776E3A092D31300A0A73706565648A
:1008C000203D2064656C7461202A206D61785F731F
:1008D00070656564202A2028726570656174202F18
:1008E0002074696D655F746F5F6D6178290A003FE0
:1008F000004D3E2000433E20004C25640A000A09BA
:100900002D20436F6E736F6C65202D0A4553432F66
:10091000713A09717569740A6D3A096D6F7573657D
:100920006B65790A000A092D204D61676963202DE6
:100930000A643A0964656275670A783A096465620F
:100940007567206D61747269780A6B3A0964656233
:100950007567206B6579626F6172640A6D3A09642C
:1009600065627567206D6F7573650A763A097665FD
:100970007273696F6E0A733A097374617475730ADE
:10098000633A09636F6E736F6C65206D6F64650AFF
:10099000302D343A096C61796572302D3428463136
:1009A000302D4634290A506175733A09626F6F74AD
:1009B0006C6F616465720A6E3A094E4B524F0A00C1
:1009C0003F004E4B524F3A206F66660A004E4B5224
:1009D0004F3A206F6E0A0074696D65725F726561CF
:1009E00064333228293A202530346C580A006B656C
:1009F00079626F6172645F6E6B726F3A2025580A7C
:100A0000006B6579626F6172645F69646C653A203E
:100A100025580A006B6579626F6172645F70726F4E
:100A2000746F636F6C3A2025580A00686F73745FA7
:100A30006B6579626F6172645F6C65647328293AD3
:100A40002025580A000A092D2053746174757320FB
:100A50002D0A004743433A20342E392E3220415686
:100A6000522D4C4942433A20312E382E3073766E47
:100A7000204156525F415243483A20617672350A0E
:100A8000004F5054494F4E533A204C554641204D4B
:100A90004F5553454B45592045585452414B4559A4
:100AA00020434F4E534F4C4520434F4D4D414E44F4
:100AB000204E4B524F204B45594D41505F534543BB
:100AC00054494F4E20343039360A004255494C447F
:100AD0003A20323232616462372D6469727479204F
:100AE0002831313A35313A34362053657020313768
:100AF0002032303136290A005649443A20307846AF
:100B000045454428742E6D2E6B2E29205049443AB9
:100B1000203078363531322850532F32206B6579AA
:100B2000626F61726420636F6E766572746572299C
:100B3000205645523A203078303030310A00444552
:100B400053433A20636F6E766572742050532F3290
:100B5000206B6579626F61726420746F2055534217
:100B60000A000A092D2056657273696F6E202D0ADE
:100B7000000A6D6F7573653A206F66660A000A6D2C
:100B80006F7573653A206F6E0A000A6B6579626F44
:100B90006172643A206F66660A000A6B6579626F5B
:100BA0006172643A206F6E0A000A6D61747269782E
:100BB0003A206F66660A000A6D61747269783A209D
:100BC0006F6E0A000A64656275673A206F6E0A00EC
:100BD0000A64656275673A206F66660A000A0A62EF
:100BE0006F6F746C6F616465722E2E2E2000433E11
:100BF000200011241FBECFEFDAE0DEBFCDBF04B668
:100C000003FE27C08091600290916102A091620270
:100C1000B09163028730904BA740B04BD1F4109253
:100C2000600210926102109262021092630214BE7E
:100C300084B7877F84BF0FB6F894A8958091600031
:100C4000886180936000109260000FBEE0E0F8E3DE
:100C5000099511E0A0E0B1E0ECEBF3E502C00590EE
:100C60000D92A634B107D9F722E0A6E4B1E001C0A5
:100C70001D92A036B207E1F70E94ED0C0C94DC291E
:100C80000C940000FF93EF93E0914601F09147012F
:100C9000309709F00995EF91FF910895FC01859136
:100CA000803011F0EFDFFBCF0895FF27E0E230E264
:100CB00047FF0CC0419597FF09C0EDE26095709524
:100CC00080959095611D711D811D911D27FF02C0AA
:100CD000219530E350E2AA27660F771F881F991FDE
:100CE000AA1FA41710F0A41B63955A95A9F7AA3060
:100CF00008F0A95FA05DAF93F395611571058105BB
:100D0000910541F7ED3211F4EF93F395F21718F4D2
:100D10003F93F395FBCF8F91B5DFFA95E1F70895F7
:100D2000E991F9918591803021F0853219F0AADF9F
:100D3000F9CF089520E0E89455915532C1F350332E
:100D400011F4689455915A3348F4505390F3220F9C
:100D5000022E220F220F200D250FF4CF0EF4219525
:100D600089919991533619F3533729F1533559F134
:100D7000BC0188279927E8945C3621F489919991E0
:100D800068945591543639F446EF7EF077FF0DC0E4
:100D90008FEF9FEF0AC055374AE039F0583540E1F0
:100DA00021F0523642E009F00895FF93EF937DDF82
:100DB000EF91FF91B7CFFF93EF93FC0181918030CA
:100DC000B9F360DFFBCFFF93EF9368DFF1CFDF93E1
:100DD000CF93CDB7DEB72596A3DFCF91DF910895EE
:100DE000E82FE695E695E695F0E0E65BFE4F40815C
:100DF000282F277081E090E002C0880F991F2A9564
:100E0000E2F7242F30E028233923232B29F4842BE5
:100E1000808381E0809349010895E82FE695E69567
:100E2000E695F0E0E65BFE4F2081382F377081E0D9
:100E300090E002C0880F991F3A95E2F7422F50E0E8
:100E400048235923452B31F080958223808381E00C
:100E5000809349010895EAE4F1E080E28E0F119257
:100E60008E13FDCF089580913D02816080933D02F5
:100E70000E94D908EAE4F1E080E28E0F11928E130D
:100E8000FDCF0895CF93109249018091690186FFAB
:100E900003C08EEF0E940D070E94D409C82F88233B
:100EA00061F01F928F9381EE92E09F938F930E9447
:100EB000E7060F900F900F900F9080918C01811199
:100EC000E1C0E09148018E2F90E08E30910508F04E
:100ED000D7C0FC01EA5AFF4F0C94F726CA3A31F109
:100EE00078F4C338F9F0C438F9F0C11134C00E9465
:100EF0002B070E94901788ED92E00E944E06C0C01A
:100F0000C13E71F020F4C03E31F582E092C0C03F96
:100F100029F0CC3F01F587E191E00AC081E089C06A
:100F200084E087C083E8AAC08CEFA8C084E191E088
:100F30009F938F938AE191E09F938F930E94112753
:100F40000E9404120E949108109248010F900F9085
:100F50000F900F9097C0C7FD02C08C2F8FC00E94CA
:100F60002B070E9490171F92CF9384EB92E09F93E0
:100F70008F930E94E7060F900F900F900F9080C004
:100F8000C93509F47DC020F4C23109F479C008C024
:100F9000CE3721F0C03F21F483E04BC08BE049C045
:100FA000C7FD03C08C2F806869C00E942B070E9478
:100FB00090171F92CF9382E992E0D9CFC43831F0D5
:100FC000C03F31F0C33889F483E824C08CEF22C0DD
:100FD0000E942B070E94901781E692E09F938F93C7
:100FE0000E94E7060F900F904DC0C7FD02C08C2FE6
:100FF00011C00E942B070E9490171F92CF938FE37E
:1010000092E0B5CFC231E1F1C935D1F1C7FD05C0DC
:101010008C2F80680E940D0733C00E942B070E940E
:1010200090171F92CF938AE192E0A1CFC43141F58E
:1010300085E08093480126C0C73711F586E0F9CFD7
:10104000C13EF1F487E0F5CFC03FD1F488E0F1CFA5
:10105000C431B1F489E0EDCFC03F91F48AE0E9CF2B
:10106000C73771F40AC0C03E59F48CE0E2CFC03FEC
:1010700039F48DE0DECFCE3719F48EEF0E94F00602
:101080001092480181E0CF910895E82FF0E0E65BEF
:10109000FE4F80810895CF92DF92EF92FF920F93DF
:1010A0001F93CF93DF938BE092E00E944E068AE479
:1010B000E82E81E0F82EC0E0D0E096E0C92E92E064
:1010C000D92E0EEF11E0DF93CF93DF92CF920E94E3
:1010D000E70683E092E00E944E06F70181917F01CE
:1010E0000E94C51D1F928F931F930F930E94E706C6
:1010F0008CEF91E00E944E0621968DB79EB7089620
:101100000FB6F8949EBF0FBE8DBFC032D105D9F681
:10111000DF91CF911F910F91FF90EF90DF90CF90D3
:101120000895982F82FB882780F990FD826091FDB9
:1011300084600C943C0A9FB7F89420916A018091D6
:101140006B01821761F030E0F901E459FE4F8081B4
:101150002F5F3F4F2F71332720936A0101C080E03A
:101160009FBF0895CF93DF93EC010E944B0A882321
:1011700041F0209731F085E08A95F1F70000219742
:10118000F4CFCE01DF91CF910895CF93DF93C2E3E7
:10119000D0E00E944B0A811108C0209731F085E011
:1011A0008A95F1F700002197F4CFCE01DF91CF911E
:1011B00008950E94480A0E94590A5598529886E755
:1011C0008093CA001092C8001092CD001092CC00FB
:1011D00080E98093C90008958AE1815011F40C944C
:1011E0009B083FB7F89420916B0190916A013FBF33
:1011F0002913F5CFEFE9FFE03197F1F700C00000C8
:10120000ECCFEF92FF920F931F93CF93DF93E82ED3
:1012100010928C011092CA008091C900877E809341
:10122000C9000E94450A0E94590A8FE891E001977F
:10123000F1F700C000000E94560A0E94480A80E1AF
:1012400097E20E94B208892B11F48AE077C0C0E0CF
:10125000D0E011E0F12C01E090E59A95F1F7C7019B
:101260000C2E02C0959587950A94E2F780FF04C082
:1012700010270E94590A02C00E94560A0E94C508FF
:10128000892B11F482E05AC082E390E00E94B208F8
:10129000892B11F483E052C02196C830D105E1F6C4
:1012A00080E58A95F1F7112319F00E94590A02C0CE
:1012B0000E94560A0E94C508892B11F484E03EC0A2
:1012C00082E390E00E94B208892B11F485E036C0D9
:1012D00090E59A95F1F70E94590AC2E3D0E00E9486
:1012E0005C0A882341F0209741F025E02A95F1F728
:1012F00000002197F4CFCD2B11F486E01FC082E3CC
:1013000090E00E94B208892B11F487E017C00E9478
:10131000C508892B11F488E011C0C2E3D0E00E9417
:101320005C0A811108C0209741F085E08A95F1F7A9
:1013300000002197F4CFCD2BE9F489E080938C0154
:101340000E94480A0E94590A5598529886E780934D
:10135000CA001092C8001092CD001092CC0080E913
:101360008093C90080E0DF91CF911F910F91FF9092
:10137000EF9008950E94480A0E94590A5598529881
:1013800086E78093CA001092C8001092CD00109298
:10139000CC0080E98093C900DF91CF911F910F911C
:1013A000FF90EF900C94EC082FB7F89490916B019C
:1013B00080916A012FBF981721F010928C010C9434
:1013C0009B0880E280938C0180E008951F920F9229
:1013D0000FB60F9211242F933F934F935F936F9308
:1013E0007F938F939F93AF93BF93CF93EF93FF938D
:1013F0008091C8008C714091CE0081111BC0CFB785
:10140000F89480916B0190E09C012F5F3F4F2F710A
:10141000332750916A01521739F0FC01E459FE4F0D
:10142000408320936B0104C086EE92E00E944E063A
:10143000CFBF10C01F924F931F928F9382EF92E005
:101440009F938F930E94E7060F900F900F900F903D
:101450000F900F90FF91EF91CF91BF91AF919F911E
:101460008F917F916F915F914F913F912F910F904D
:101470000FBE0F901F901895CF93C82F8DEE0E942E
:1014800001098C2FCF910C9401095D98559A08950C
:1014900055985D9A089555985D9A85E08A95F1F77B
:1014A000000089B185FB882780F908955A98529ADF
:1014B000089552985A9A089552985A9A85E08A95B2
:1014C000F1F7000089B182FB882780F908958091A7
:1014D000B10108959FB7F894109290019FBF909129
:1014E0005102943009F057C09091E9009F703091FB
:1014F000EC00232F217030FD20E8922B24E0209374
:10150000E9002091EB0020FF43C02091EE0027FF6F
:101510003FC020918D01222321F02091E80025FF7A
:1015200037C010928D0126E03091E80035FD15C0DE
:1015300030915102343061F53091EB0035FD28C017
:10154000215021F481E080938D0122C0EFE9FFE07A
:101550003197F1F700C00000E7CF8093F100809150
:10156000E80085FD0AC08091E80080FFFCCF8091F3
:10157000E8008E778093E80006C08FB7F89421E0EA
:10158000209390018FBF9F709093E90080E00895B1
:101590009F709093E9008FEF0895CF93DF9300D071
:1015A0001F92CDB7DEB79C0180915102843019F5AE
:1015B00093E099833B832A839093E9008FEF909186
:1015C000E800815095FD06C095ED9A95F1F7000071
:1015D0008111F5CF8091E80085FF0DC040E050E01B
:1015E00063E070E0CE0101960E94B40D8091E800A6
:1015F0008E778093E8000F900F900F90DF91CF913E
:101600000895CF93DF9300D01F92CDB7DEB720911E
:101610005102243021F522E029839B838A8383E0D1
:101620008093E9008FEF9091E800815095FD06C00E
:1016300095ED9A95F1F700008111F5CF8091E800C2
:1016400085FF0DC040E050E063E070E0CE01019600
:101650000E94B40D8091E8008E778093E8000F908F
:101660000F900F90DF91CF91089520915102243077
:10167000F1F422E02093E9002FEF3091E8002150AF
:1016800035FD06C035ED3A95F1F700002111F5CF93
:101690002091E80025FF0BC040E050E065E070E0DD
:1016A0000E94B40D8091E8008E778093E800089541
:1016B000CF93DF9320915102243009F048C0EC0110
:1016C00080910A018823E1F080910B018823C1F009
:1016D00085E08093E9008FEF9091E800815095FDBF
:1016E00006C095E19A95F1F700008111F5CF809140
:1016F000E80085FF2CC040E050E060E270E017C0D9
:1017000081E08093E9008FEF9091E800815095FD92
:1017100006C095ED9A95F1F700008111F5CF809103
:10172000E80085FF14C040E050E068E070E0CE01C2
:101730000E94B40D8091E8008E778093E80080E2EB
:10174000FE01A1E9B1E001900D928A95E1F7DF91E8
:10175000CF91089582E493E00E944E06809150025A
:10176000811109C00E944B0F0E94A80F8091E200D6
:1017700084608093E20008958EE393E00E944E0619
:10178000109250020895089520918E012F5F822FAC
:1017900062E30E94D726992319F020938E010895C1
:1017A00010928E0180919001882371F180915102F5
:1017B000843041F58091E9008F702091EC00922FE8
:1017C000917020FD90E8892B94E09093E90090912E
:1017D000EB0090FF14C09091EE0097FF10C0909125
:1017E000E80095FF03C01092F100F9CF9091E80056
:1017F00090FF05C09091E8009E779093E8008F706D
:101800008093E90010929001089542E061EC81E03C
:101810000E94C50E42E061EC82E00E94C50E42E0EB
:1018200061EC83E00E94C50E42E261EC84E00E941C
:10183000C50E42E261EC85E00C94C50E8091530226
:10184000833009F455C030F4813071F0823009F4EE
:101850008EC008958A3009F47AC08B3009F460C0D4
:10186000893009F09CC020C080915202813A09F071
:1018700096C08091E800877F8093E80080915602AF
:1018800090915702892B21F460E281E991E003C035
:1018900060E080E090E070E00E94010E8091E8003E
:1018A0008B778093E800089580915202813209F08D
:1018B00076C08091560290915702009719F00497D4
:1018C00009F06DC08091E800877F8093E8008091E7
:1018D000E80082FD05C0809151028111F8CF5FC000
:1018E0008091F1008093B1018091E8008B7753C023
:1018F00080915202813A09F052C080915602909133
:101900005702892B09F04BC08091E800877F8093B4
:10191000E8008091E80080FFFCCF80910A0136C08A
:10192000809152028132D9F58091560290915702EE
:10193000892BA9F58091E800877F8093E8000E94B9
:10194000FA0E8091540280930A010C9490178091B2
:101950005202813221F58091E800877F8093E80070
:101960000E94FA0E809155028093B20108958091F1
:101970005202813AA1F48091E800877F8093E800C9
:101980008091E80080FFFCCF8091B2018093F1004C
:101990008091E8008E778093E8000C94FA0E089509
:1019A000089508958091B10180938F011092B10143
:1019B00080E00E9491080E9433070C9490170C94C9
:1019C000D20C0E94EF1D80914F02882329F00E94C3
:1019D000FE1D81110C949E0D089584B7877F84BFEE
:1019E0000FB6F894A895809160008861809360009C
:1019F000109260000FBE90E080E80FB6F8948093DC
:101A00006100909361000FBE8AE69AE00E94C01DBB
:101A100086E393E00E944E060E94D00C0E94911231
:101A20000E944B0F0E94A80F8091E2008460809377
:101A3000E200789480915102843019F00E94E41100
:101A4000F9CF85E293E00E944E060E94931280E057
:101A500091E00E94FF1184E193E00E944E060E94F3
:101A6000D10C80915102853019F40E94E10CF9CF1C
:101A70000E9497120E94E411F4CF0E94121E8091DE
:101A80008F018093B10108950C943D0D292F3327C8
:101A900023303105C9F064F42130310581F0223062
:101AA000310509F043C08DE890E02CE833E042C0F6
:101AB00021323105F1F02232310541F137C082E1A6
:101AC00090E029E134E036C099278130910541F05A
:101AD0008230910541F0892B49F5E8E8F3E005C033
:101AE000E8E7F3E002C0E6E4F3E0849190E09F01D0
:101AF00021C06530D8F4E62FF0E0EE0FFF1FEF5C59
:101B0000FE4F2081318189E090E014C0653070F48F
:101B100070E0FB01EE0FFF1FE95DFE4F2081318178
:101B2000FB01EE5DFE4F808190E004C080E090E01C
:101B300020E030E0FA0131832083089580E189BDFF
:101B400082E189BD09B400FEFDCF8091D8008F7D70
:101B50008093D8008091E00082608093E0008091C3
:101B6000E00081FDFCCF0895CF92DF92EF92FF92CB
:101B70000F931F93CF93DF93EC018B017A010E94A7
:101B8000190F811135C0E114F10439F0F70180819A
:101B90009181081B190BC80FD91FC12CD12C01151D
:101BA000110529F18091E80085FD18C08091E800B9
:101BB0008E778093E8000E94E411E114F10449F06B
:101BC000F70180819181C80ED91ED182C08285E043
:101BD0000FC00E94190F882311F30AC089918093C6
:101BE000F10001501109FFEFCF1ADF0AD8CF80E0D2
:101BF000DF91CF911F910F91FF90EF90DF90CF90E9
:101C0000089520915802309159022617370748F05D
:101C10006115710539F42091E8002E772093E800D2
:101C200001C0B90140E061157105A9F1209151028F
:101C3000222309F443C0253009F442C02091E80072
:101C400023FD40C02091E80022FD32C02091E80031
:101C500020FFE9CF4091F3002091F20030E0342BD7
:101C6000FC01CF016115710559F02830310540F4B0
:101C700081918093F100615071092F5F3F4FF1CF47
:101C800041E02830310509F040E02091E8002E774E
:101C90002093E800C8CF4111C9CF0AC080915102FA
:101CA000882361F0853061F08091E80083FD0AC0EF
:101CB0008091E80082FFF2CF80E0089582E00895ED
:101CC00083E0089581E008952091580230915902EF
:101CD0002617370748F06115710539F42091E8009F
:101CE0002E772093E80001C0B901FC0120E06115C6
:101CF000710591F180915102882309F440C085302B
:101D000009F43FC08091E80083FD3DC08091E80068
:101D100082FD2FC08091E80080FFE9CF2091F30081
:101D20008091F20090E0922B6115710559F0883096
:101D3000910540F424912093F1003196615071098E
:101D40000196F2CF21E0089709F020E08091E800A9
:101D50008E778093E800CBCF2111CCCF0AC0809141
:101D60005102882361F0853061F08091E80083FDA5
:101D70000AC08091E80082FFF2CF80E0089582E0FF
:101D8000089583E0089581E00895982F973058F5DD
:101D90009093E900981739F07091EC002091ED00D4
:101DA0005091F00003C0242F762F50E021FF19C07E
:101DB0003091EB003E7F3093EB003091ED003D7FA2
:101DC0003093ED003091EB0031603093EB00709375
:101DD000EC002093ED005093F0002091EE0027FFDF
:101DE00007C09F5FD3CF8F708093E90081E0089593
:101DF00080E008958091520287FF11C08091E80031
:101E000082FD05C0809151028111F8CF11C08091EF
:101E1000E8008B770BC080915102882349F08091B4
:101E2000E80080FFF8CF8091E8008E778093E8008B
:101E300008952091E4003091E50095E64091EC0092
:101E4000842F817040FF22C08091E80080FD1CC07B
:101E500080915102882391F0853091F08091EB00C0
:101E600085FD10C04091E4005091E50042175307F2
:101E700029F39A01915011F784E0089582E00895C2
:101E800083E0089581E0089580E008954091E8009E
:101E900042FFDECF08950E94B90F0E94C10FE0EE0D
:101EA000F0E0808181608083E8EDF0E080818F77D1
:101EB000808319BCA7EDB0E08C918E7F8C938081DC
:101EC0008F7E80831092500208950F931F93CF93BB
:101ED000DF930E94B90F0E94C10FC8EDD0E0888146
:101EE0008F77888388818068888388818F7D8883C5
:101EF00019BC1092510210924D0210924F02109292
:101F00004E0200EE10E0F80180818B7F8083888193
:101F10008160888342E060E080E00E94C50EE1EECF
:101F2000F0E080818E7F8083E2EEF0E0808181604E
:101F30008083808188608083F80180818E7F8083A8
:101F4000888180618883DF91CF911F910F910895DF
:101F5000E8EDF0E080818F7E8083E7EDF0E0808126
:101F60008160808384E082BF81E0809350020C9482
:101F7000650FE8EDF0E080818E7F80831092E200B3
:101F800008951092DA001092E10008951F920F92C6
:101F90000FB60F9211242F933F934F935F936F933C
:101FA0007F938F939F93AF93BF93EF93FF93809112
:101FB000E10082FF0BC08091E20082FF07C08091A8
:101FC000E1008B7F8093E1000E94C40B8091DA00D6
:101FD00080FF1FC08091D80080FF1BC08091DA0075
:101FE0008E7F8093DA008091D90080FF0DC080E160
:101FF00089BD82E189BD09B400FEFDCF81E08093F7
:1020000051020E94AA0B05C019BC109251020E94F5
:10201000BC0B8091E10080FF19C08091E20080FF3D
:1020200015C08091E2008E7F8093E2008091E200F3
:1020300080618093E2008091D80080628093D80014
:1020400019BC85E0809351020E94DF0C8091E10071
:1020500084FF30C08091E20084FF2CC080E189BD04
:1020600082E189BD09B400FEFDCF8091D8008F7D4B
:102070008093D8008091E1008F7E8093E100809171
:10208000E2008F7E8093E2008091E2008160809385
:10209000E20080914D02882311F084E007C0809116
:1020A000E30087FD02C081E001C083E0809351021C
:1020B0000E94440D8091E10083FF24C08091E200E2
:1020C00083FF20C08091E100877F8093E10082E060
:1020D0008093510210924D028091E1008E7F809397
:1020E000E1008091E2008E7F8093E2008091E20027
:1020F00080618093E20042E060E080E00E94C50ED3
:102100000E94C30BFF91EF91BF91AF919F918F916F
:102110007F916F915F914F913F912F910F900FBEE3
:102120000F901F9018951F93CF93DF93CDB7DEB715
:10213000AA970FB6F894DEBF0FBECDBFE2E5F2E07E
:1021400088E08E0F9091F10091938E13FBCF0E9447
:102150001E0C8091E80083FF1FC180915202909174
:102160005302492F50E04A30510508F015C1FA01D9
:10217000EC59FF4F0C94F726803881F0823809F033
:102180000BC1809156028F708093E9008091EB0023
:1021900085FB882780F91092E90006C080914E02E5
:1021A00090914F02911182609091E800977F9093F7
:1021B000E8008093F1001092F100C8C0282F2D7F15
:1021C00009F0EAC0882319F0823061F0E5C08091FF
:1021D0005402813009F0E0C0933009F080E0809330
:1021E0004F022BC080915402811127C0809156026A
:1021F0008F7009F4D1C08093E9002091EB0020FF9B
:102200001CC0933021F48091EB00806214C0909147
:10221000EB0090619093EB0021E030E0A90102C057
:10222000440F551F8A95E2F74093EA001092EA00A6
:102230008091EB0088608093EB001092E900809120
:10224000E800877F86C08111A7C0109154021F77D4
:102250008091E3008078812B8093E3008091E800F7
:10226000877F8093E8000E94FA0E8091E80080FF4B
:10227000FCCF8091E30080688093E300111102C0DD
:1022800082E001C083E08093510286C08058823092
:1022900008F082C080915402909155028C3D53E029
:1022A000950779F583E08A838AE289834FB7F894AA
:1022B000DE01139620E03EE051E2E32FF0E0509380
:1022C0005700E49120FF03C0E295EF703F5FEF708D
:1022D0008E2F90E0EA3010F0C79601C0C0968D9323
:1022E0009D932F5F243149F74FBF8091E800877F8E
:1022F0008093E8006AE270E0CE0101960E94010E30
:1023000014C0AE014F5F5F4F609156020E94460DB0
:10231000BC01892B09F440C09091E800977F90930D
:10232000E80089819A810E94640E8091E8008B7791
:102330008093E80031C0803879F58091E800877F8C
:102340008093E80080914D028093F1008091E80035
:102350008E778093E8000E94FA0E1EC081111CC087
:10236000909154029230C0F48091E800877F80936E
:10237000E80090934D020E94FA0E80914D02811167
:1023800006C08091E30087FD02C081E001C084E0C7
:10239000809351020E94050C8091E80083FF0AC0DF
:1023A0008091E800877F8093E8008091EB00806255
:1023B0008093EB00AA960FB6F894DEBF0FBECDBF98
:1023C000DF91CF911F910895CF938091510288237F
:1023D000A1F0C091E900CF709091EC00892F81703D
:1023E00090FD80E8C82B1092E9008091E80083FD01
:1023F0000E949310CF70C093E900CF9108959093FD
:10240000B8018093B7010895E091B701F091B80148
:10241000309721F00190F081E02D099480E008953B
:10242000EF92FF920F931F93CF93DF93E091B70149
:10243000F091B8013097B1F18C010280F381E02D69
:10244000099580913D0282FF2DC080FF04C081E587
:1024500095E00E944E06E80110E28BE4E82E85E04C
:10246000F82E80913D0280FF0BC088811F928F93D0
:10247000FF92EF920E94E7060F900F900F900F903F
:10248000115021961111EDCF80913D0280FF0AC0BD
:1024900089E495E0DF91CF911F910F91FF90EF902C
:1024A0000C944E06DF91CF911F910F91FF90EF900A
:1024B0000895E091B701F091B801309721F00480C0
:1024C000F581E02D099408952091B5013091B60170
:1024D0008217930771F09093B6018093B501E09154
:1024E000B701F091B801309721F00680F781E02D17
:1024F000099408952091B3013091B4018217930794
:1025000071F09093B4018093B301E091B701F09121
:10251000B801309721F00084F185E02D09940895E9
:1025200008950C9490120E943B1E0C943307CF9296
:10253000DF92EF92FF920F931F93CF93DF9300D020
:1025400000D000D0CDB7DEB70E9442078AEBC82E7C
:1025500081E0D82E00E010E0E02E802F0E94450898
:10256000F60141916F01F42EF826B1F40F5F1F4F71
:102570000032110589F78FEF89838A831B820E94BD
:10258000441E8160782F9D838C8349815A816B81A1
:102590008D810E94561347C090913D0291FF04C067
:1025A0008E830E944B088E8120E030E04F2D50E05A
:1025B000922FBA01022E02C0759567950A94E2F730
:1025C00060FF2BC02983EA8221E030E0690102C06C
:1025D000CC0CDD1C9A95E2F790E08C219D21892B93
:1025E00009F420E02B830E94441E8160782F9D8394
:1025F0008C8349815A816B818D810E945613498158
:102600005A816B817C818D810E94DC1DF801E6542A
:10261000FE4F8081C826C08206C02F5F3F4F283002
:10262000310531F6A3CF0E94DB1D0E9405211091D8
:10263000B9010E940412181741F10E9404128093FC
:10264000B90190913D0292FF0EC090FF0CC01F9205
:102650008F9383E695E09F938F930E94E7060F90F8
:102660000F900F900F908091B90126960FB6F894B5
:10267000DEBF0FBECDBFDF91CF911F910F91FF90B5
:10268000EF90DF90CF900C94ED1D26960FB6F89446
:10269000DEBF0FBECDBFDF91CF911F910F91FF9095
:1026A000EF90DF90CF9008950C949108CF93DF9333
:1026B000CDB7DEB72B970FB6F894DEBF0FBECDBFF8
:1026C000942F4F83252F588769877A878B874A8570
:1026D0005B85452B21F02F3F09F59F3FF9F4DE0183
:1026E000119686E0FD0111928A95E9F785E0FE01D9
:1026F000379601900D928A95E1F749815A816B8155
:102700007C818D819E810E942A1A2B960FB6F894A7
:10271000DEBF0FBECDBFDF91CF9108954F815885A9
:1027200069857A858B850E94DC1DD9CFCF9388235C
:1027300009F4A4C0C82F8CEF8C0F813A48F48C2F79
:102740000E944F2481119AC08C2F0E94B51C0CC08E
:1027500080E28C0F883058F4C77081E001C0880F88
:10276000CA95EAF70E94601DCF910C949A1D8BE5E3
:102770008C0F833078F4C53A29F0C63A31F083E8FB
:1027800090E005C081E890E002C082E890E0CF913F
:102790000C94641288E58C0F853108F06FC0C83A3C
:1027A00061F1C93A69F1CA3A71F1CB3A79F1CC3A9F
:1027B00081F1CD3A89F1CE3A91F1CF3A99F1C13B0D
:1027C000A1F1C03BA9F1C23BB1F1C33BB9F1C43B9C
:1027D000C1F1C53BC9F1C63BD1F1C73BD9F1C83BFB
:1027E000E1F1C93BE9F1CA3BF1F1CB3BF9F1CC3B5B
:1027F00009F43FC080E090E03EC082EE90E03BC034
:1028000089EE90E038C08AEE90E035C085EB90E02C
:1028100032C086EB90E02FC083EB90E02CC084EBBD
:1028200090E029C087EB90E026C08CEC90E023C0BC
:102830008DEC90E020C083E891E01DC08AE891E033
:102840001AC082E991E017C084E991E014C081E2E6
:1028500092E011C083E292E00EC084E292E00BC0ED
:1028600085E292E008C086E292E005C087E292E04D
:1028700002C08AE292E0CF910C947A12CF9108952F
:10288000882329F19CEF980F913A18F40E94081DB3
:102890000DC090E2980F983058F4877091E001C015
:1028A000990F8A95EAF7892F0E94661D0C949A1D4C
:1028B0009BE5980F933020F480E090E00C94641234
:1028C000885A853120F480E090E00C947A120895C3
:1028D000882321F00E94601D0C949A1D089588237E
:1028E00021F00E94661D0C949A1D0895CF92DF92EC
:1028F000EF92FF920F931F93CF93DF9300D000D0FE
:1029000000D0CDB7DEB725E0FC01DE0111960190C5
:102910000D922A95E1F7FC0140813181F2802581F9
:1029200022952F7063817481672B09F4D8C23F3FD1
:1029300019F44F3F09F4D3C26C0149833A8389816A
:102940009A812E830E94741C182F092F0E94731CD9
:102950000E94831BE02FE295EF70F0E0E259FF4FF9
:102960002E810C94F726802F807F902F9F70092F47
:10297000882311F00295007FFF2049F0002309F41D
:102980005FC2802F0E94731D0E949A1D59C2812F21
:102990000E944014002309F4A2C2802F0E94791DD6
:1029A00026960FB6F894DEBF0FBECDBFDF91CF9154
:1029B0001F910F91FF90EF90DF90CF900C949A1D94
:1029C000802F807F902F9F70092F803211F0029509
:1029D000007F112319F0113001F129C0FF20A9F067
:1029E000802F222349F1213039F526960FB6F8942D
:1029F000DEBF0FBECDBFDF91CF911F910F91FF9032
:102A0000EF90DF90CF900C94831D222319F021309A
:102A100009F465C20E94861D2CC0FF20E9F0263013
:102A200008F05DC20E945D1D802329F022C0FF20B6
:102A3000F1F0211115C0802F26960FB6F894DEBF55
:102A40000FBECDBFDF91CF911F910F91FF90EF90FF
:102A5000DF90CF900C946814253008F040C209C074
:102A6000F601858180FFECC18F708583E4CF211151
:102A7000FBC1802F69C1202F26952695237030E059
:102A80002115310521F021303105C9F028C2FF2080
:102A900021F0812F902F937002C080E090E0269665
:102AA0000FB6F894DEBF0FBECDBFDF91CF911F915F
:102AB0000F91FF90EF90DF90CF900C946412FF2065
:102AC00021F0812F902F937002C080E090E0269635
:102AD0000FB6F894DEBF0FBECDBFDF91CF911F912F
:102AE0000F91FF90EF90DF90CF900C947A12812F8E
:102AF000FF2019F00E948B1F02C00E94F31F269630
:102B00000FB6F894DEBF0FBECDBFDF91CF911F91FE
:102B10000F91FF90EF90DF90CF900C947820802F52
:102B2000837009F078C0F110DAC1812F8295869503
:102B30008770880F880F912F9F70C92ED12CE12CA0
:102B4000F12C082E04C0CC0CDD1CEE1CFF1C0A94DA
:102B5000D2F714FF12C04FE050E060E070E004C014
:102B6000440F551F661F771F8A95D2F7CB01BA0114
:102B7000609570958095909503C060E070E0CB0102
:102B8000202F269526952370422F50E04230510584
:102B9000D1F04330510559F16C297D298E299F29A7
:102BA0004130510541F126960FB6F894DEBF0FBEB5
:102BB000CDBFDF91CF911F910F91FF90EF90DF90EC
:102BC000CF900C94981B6C297D298E299F292696DD
:102BD0000FB6F894DEBF0FBECDBFDF91CF911F912E
:102BE0000F91FF90EF90DF90CF900C94AA1B0E9462
:102BF000981BC701B60126960FB6F894DEBF0FBE2C
:102C0000CDBFDF91CF911F910F91FF90EF90DF909B
:102C1000CF900C94861BFF2019F0802F817001C08B
:102C20008695882309F45BC1812F829586958770EC
:102C3000880F880F912F9F70C92ED12CE12CF12C79
:102C4000082E04C0CC0CDD1CEE1CFF1C0A94D2F72D
:102C500014FF12C04FE050E060E070E004C0440F89
:102C6000551F661F771F8A95D2F7CB01BA01609571
:102C700070958095909503C060E070E0CB01202FA7
:102C8000269526952370422F50E042305105D1F011
:102C90004330510559F16C297D298E299F294130F6
:102CA000510541F126960FB6F894DEBF0FBECDBF99
:102CB000DF91CF911F910F91FF90EF90DF90CF9018
:102CC0000C944F1C6C297D298E299F2926960FB6BE
:102CD000F894DEBF0FBECDBFDF91CF911F910F9152
:102CE000FF90EF90DF90CF900C94611C0E944F1CDE
:102CF000C701B60126960FB6F894DEBF0FBECDBF52
:102D0000DF91CF911F910F91FF90EF90DF90CF90C7
:102D10000C943D1C103F41F118F4103E48F48BC058
:102D2000123F09F450C0D8F1133F09F460C083C0CA
:102D30001F70802F8F71FF2021F00E94D61B812FE2
:102D40007BCE0E94F71B812F26960FB6F894DEBF2C
:102D50000FBECDBFDF91CF911F910F91FF90EF90EC
:102D6000DF90CF900C946F14FF20A9F0253008F06D
:102D7000B6C0802F8F7126960FB6F894DEBF0FBEB7
:102D8000CDBFDF91CF911F910F91FF90EF90DF901A
:102D9000CF900C941C1C263008F0A1C0EACFFF2075
:102DA000A1F0802F8F7126960FB6F894DEBF0FBE6C
:102DB000CDBFDF91CF911F910F91FF90EF90DF90EA
:102DC000CF900C94D61BFF2061F3802F8F71269635
:102DD0000FB6F894DEBF0FBECDBFDF91CF911F912C
:102DE0000F91FF90EF90DF90CF900C94F71BFF2096
:102DF00091F0802F8F7126960FB6F894DEBF0FBE2C
:102E0000CDBFDF91CF911F910F91FF90EF90DF9099
:102E1000CF900C94C11B26960FB6F894DEBF0FBE60
:102E2000CDBFDF91CF911F910F91FF90EF90DF9079
:102E3000CF900C94BC1BFF20A1F0222309F4B1CF4A
:102E4000812F26960FB6F894DEBF0FBECDBFDF915F
:102E5000CF911F910F91FF90EF90DF90CF900C9446
:102E60009613222309F4B1CF812F26960FB6F8943A
:102E7000DEBF0FBECDBFDF91CF911F910F91FF90AD
:102E8000EF90DF90CF900C944014402F4F70612F43
:102E9000C6010E94051F26960FB6F894DEBF0FBE2E
:102EA000CDBFDF91CF911F910F91FF90EF90DF90F9
:102EB000CF900C94CE1A402F4F70612FC6012696EA
:102EC0000FB6F894DEBF0FBECDBFDF91CF911F913B
:102ED0000F91FF90EF90DF90CF900C94081F2696F3
:102EE0000FB6F894DEBF0FBECDBFDF91CF911F911B
:102EF0000F91FF90EF90DF90CF9008950E94801D7A
:102F00000E944F1D0E949A1D0E94AA210E947820B3
:102F100080E090E00E94641280E090E00C947A12CD
:102F20000E94701D0C947E170E94741C292F2295FC
:102F30002F7030E02C3031054CF42A3031056CF420
:102F4000225031092230310588F407C02C30310578
:102F500049F02F30310531F009C0803E48F0803F04
:102F600029F406C093FB882780F9089580E008952E
:102F700081E00895CF93DF9300D000D01F92CDB7AA
:102F8000DEB70F900F900F900F900F90DF91CF91C1
:102F90000895CF93DF9300D000D000D0CDB7DEB737
:102FA00026960FB6F894DEBF0FBECDBFDF91CF914E
:102FB00008951F93CF93DF93C091DA0116E08091BB
:102FC000DB01C81799F0D0E01C9FF0011D9FF00DA8
:102FD0001124E452FE4F40815181628173818481CA
:102FE00095810E94C9172196C770E9CFDF91CF91D3
:102FF0001F91089540910C0250910D0260910E02B4
:1030000070910F0280911002909111020C94C917D7
:103010008091110282958F7009F054C080910E0248
:10302000882309F44FC08091DA01A091DB016091FF
:103030000C0270910D0240910F0250911002B6E007
:103040008A1709F43FC090E041155105C1F17F3F57
:1030500011F46F3FA1F1B89FF001B99FF00D112459
:10306000E452FE4F218172132AC02081621327C0CF
:103070002281211124C0238134812417350710F4C3
:1030800021503109241B350B283C3105C0F4209117
:1030900011022F7020612093110226E0289FF00179
:1030A000299FF00D1124EF51FE4F80818F708061B8
:1030B00080838CE092E00E9476140C94D9170196DC
:1030C0008770BECF0895CF92DF92EF92FF920F9359
:1030D0001F93CF93DF93CDB7DEB762970FB6F89407
:1030E000DEBF0FBECDBF8C0185E0F801DE011D966D
:1030F00001900D928A95E1F7D8014C9111965C915F
:10310000119712966C9112971396CD90DC901497AC
:1031100030910C0270910D0280910F02909110027B
:10312000009709F46BC17F3F19F43F3F09F466C172
:10313000E0900E02EE2009F4C0C020911102C816E2
:10314000D90628F0F601E81BF90BCF0104C08095E1
:1031500090958C0D9D1DFF24F394883C910578F08B
:10316000F12C207F09F0C6C07C2DD98AC88A8989B4
:103170000E94BA178CE092E00E947614B1C0822FB0
:10318000807F09F046C0751314C0341312C061115A
:1031900010C02F702061209311020E94FA178CE05A
:1031A00092E00E94761480911102D80115968C93BA
:1031B0002EC0CD2819F15F3F11F44F3FF9F0F62EE4
:1031C00061111CC08091DA012091DB0136E0821789
:1031D00009F45AC090E0389FF001399FF00D112496
:1031E000E452FE4F7181571306C07081471303C02C
:1031F0007281711103C001968770E9CFF62E6623A4
:1032000009F418C180911102816080931102F12CA0
:1032100011C1751308C0341306C0611104C0809138
:103220001102D801C3C04D875E878D859E856A8B4C
:103230000E9494176A898823E1F16623D1F12091D5
:103240001102822F82958F7090E0029774F0809126
:103250000C0290910D0298878F831986DB86CA86AF
:103260002C87CE0107960E94761486E0F801ACE028
:10327000B2E001900D928A95E1F70E9408180E9431
:10328000FA17FF24F394D6C04D875E878D859E85FF
:103290000E94741C292F22952F7030E022303105B6
:1032A0000CF0BCC09F7009F0B6C0805E883008F496
:1032B000C1C0C8010E947614E4CFC816D90608F42C
:1032C00053C0F601E81BF90BCF01883C910508F4C7
:1032D00050C0F12C7C2DD98AC88A89890E94BA17DE
:1032E000ECE0F2E086E0DF011D928A95E9F70E94AA
:1032F000FA17A0C0751314C0341312C0611110C0A6
:1033000080911102F8018583C8010E94761486E03D
:10331000ECE0F2E0DF011D928A95E9F7FE2C8AC00D
:103320004D875E878D859E856A8B0E9494176A897A
:10333000882309F4BECF662309F4BBCF2091110284
:10334000822F82958F7090E002970CF48ECF80913F
:103350000C0290910D029A8389831B82DD82CC82BC
:103360002E83CE0101967FCF809590958C0D9D1D6B
:10337000ACCFF62E662309F49CCF75132EC0341300
:103380002CC02091110220FD1FC0822F82958F70CA
:10339000D9F0D80115962C9315978F3049F08F5F8F
:1033A000982F9295907F822F8F70892B15968C93F2
:1033B000C8010E94761486E0F801ACE0B2E001900A
:1033C0000D928A95E1F793CF86E0F801ACE0B2E088
:1033D00001900D928A95E1F72DC04D875E878D850E
:1033E0009E850E949417811140CF809111028160C7
:1033F00080931102C8010E9476141CC0662309F450
:1034000058CF4D875E878D859E850E9494178823AF
:1034100009F44FCF2ACF811148CF0CC02430310599
:103420000CF047CF9F7009F440CFF8019581907F51
:1034300009F03BCF8F2D62960FB6F894DEBF0FBE1A
:10344000CDBFDF91CF911F910F91FF90EF90DF9053
:10345000CF9008951F93CF93DF93CDB7DEB72C970E
:103460000FB6F894DEBF0FBECDBF4F835887698774
:103470007A878B879C87CE0107960E9463188823E2
:1034800069F08F8198852A853B85232BF1F19F3F39
:1034900009F063C08F3F09F060C037C086E0FE01CD
:1034A0003796DE01119601900D928A95E1F76F81B2
:1034B0007885EA85FB85309741F17F3F11F46F3FB6
:1034C00021F12091DB0130E0C90101968770992735
:1034D0004091DA0150E08417950709F447C06983E9
:1034E0007A83FD83EC8396E0929FD001939FB00D89
:1034F0001124A452BE4FFE01319601900D929A956F
:10350000E1F78093DB010E94D91716E08091DA0180
:103510009091DB018917C1F1189FC00111248452D9
:103520009E4F0E946318882379F1E091DA011E9F73
:10353000F0011124E452FE4F408151816281738178
:10354000848195810E94C9178091DA0190E00196EB
:10355000877099278093DA01D9CF4F815885698583
:103560007A858B859C850E94C917CFCF0E949017C2
:103570001092DB011092DA01ECE0F2E086E0DF016C
:103580001D928A95E9F7C1CF2C960FB6F894DEBF4D
:103590000FBECDBFDF91CF911F910895DF92EF92C3
:1035A000FF920F931F93CF93DF93FC01892B09F4B4
:1035B0008AC0E12CF12CDD24D394EF012196849173
:1035C000853709F461C058F4843708F04EC0843060
:1035D00008F06AC08130D1F0823071F174C0883750
:1035E00009F45DC050F4863709F455C0873709F0F7
:1035F0006AC08E2D0E946D1D54C09CE7980F9037B5
:1036000008F061C08F770E94401450C08F010E5F98
:103610001F4FFE01849190E2980F983050F487700C
:10362000FD2D01C0FF0F8A95EAF78F2F0E94731DB1
:1036300014C00E94961313C08F010E5F1F4FFE012E
:10364000C49180E28C0F883060F4C7708D2D01C06A
:10365000880FCA95EAF70E94791D0E949A1DE80119
:1036600025C08C2F0E944014FACF9F012E5F3F4F40
:10367000FE01C491CC2369F08FE99FE00197F1F737
:1036800000C00000C150F6CF9F012E5F3F4FFE01EA
:10369000F490E9010BC00E945D1DE82E07C00E9456
:1036A000701D0E949A1D02C00E9496138F2D8823C0
:1036B00041F0EFE9FFE03197F1F700C000008150E1
:1036C000F6CFFE017ACFDF91CF911F910F91FF903E
:1036D000EF90DF9008956093160270931702809325
:1036E0001802909319020E94EB1D0C947E176093B0
:1036F00012027093130280931402909315020E9499
:10370000EC1D0C947E1708950C946B1B0F931F9364
:10371000009116021091170220911802309119029F
:10372000602B712B822B932B1F910F910C946B1B91
:103730000F931F9300911602109117022091180207
:103740003091190260237123822393231F910F91DB
:103750000C946B1B0F931F9300911602109117028C
:103760002091180230911902602771278227932730
:103770001F910F910C946B1B60E070E0CB010C94D7
:10378000771B0F931F9341E050E060E070E08A01E7
:103790009B0104C0000F111F221F331F8A95D2F70F
:1037A000C901B8011F910F910C94771B0F931F93C0
:1037B00041E050E060E070E004C0440F551F661F18
:1037C000771F8A95D2F78091120290911302A091EF
:1037D0001402B09115028A019B01082B192B2A2B88
:1037E0003B2BC901B8011F910F910C94771B0F93CC
:1037F0001F9341E050E060E070E004C0440F551FAB
:10380000661F771F8A95D2F7409550956095709501
:103810008091120290911302A0911402B0911502AE
:103820008A019B01082319232A233B23C901B801DC
:103830001F910F910C94771B0F931F9341E050E061
:1038400060E070E004C0440F551F661F771F8A9523
:10385000D2F78091120290911302A0911402B091BC
:1038600015028A019B01082719272A273B27C9012E
:10387000B8011F910F910C94771B0F931F93009128
:103880001202109113022091140230911502602B44
:10389000712B822B932B1F910F910C94771B0F93FD
:1038A0001F93009112021091130220911402309183
:1038B000150260237123822393231F910F910C948F
:1038C000771B0F931F930091120210911302209106
:1038D00014023091150260277127822793271F91C8
:1038E0000F910C94771B0895CF92DF92EF92FF9285
:1038F0000F931F93CF93DF938C01C0901602D0904B
:103900001702E0901802F0901902409112025091B3
:1039100013026091140270911502C42AD52AE62A76
:10392000F72ACFE1D0E0D701C6010C2E04C0B6952E
:10393000A795979587950A94D2F780FF07C0B8019D
:103940008C2F0E94DB1E8130910531F4219758F7AE
:10395000B80180E00E94DB1EDF91CF911F910F9193
:10396000FF90EF90DF90CF90089590910A019923F6
:1039700021F090910B01911109C020910C0130911F
:103980000D01F90132969FEF40E030C0982F9695D7
:10399000969596959F31A0F4E0910C01F0910D0160
:1039A000E90FF11D877021E030E0A90102C0440F4A
:1039B000551F8A95E2F7CA019181892B8183089569
:1039C00090913D0290FF23C01F928F938CE895E069
:1039D0009F938F930E94E7060F900F900F900F9088
:1039E00008959F3F39F04F5F4E3141F05191581388
:1039F000F8CF0DC05111F7CF942FF5CF9F3F39F07D
:103A0000F901E90FF11D97FDFA9582830895089554
:103A100090910A01992321F090910B01911109C015
:103A200020910C0130910D01F9013296205E3F4F3B
:103A300030C0982F9695969596959F31A8F4E09171
:103A40000C01F0910D01E90FF11D877021E030E0CC
:103A5000A90102C0440F551F8A95E2F7CA0180955B
:103A6000918189238183089590913D0290FF16C032
:103A70001F928F938EE695E09F938F930E94E706A7
:103A80000F900F900F900F9008953196E217F30763
:103A900029F090819813F9CF1082F7CF089581E033
:103AA00090E0E0910C01F0910D01E80FF91F1082F8
:103AB000019680329105A9F7089580913C020895FE
:103AC00090913C02892B80933C02089580959091BF
:103AD0003C02892380933C02089580933C02089520
:103AE00010923C02089590913B02892B80933B02F7
:103AF0000895809590913B02892380933B0208951D
:103B000010923B02089580931A02089510921A02AF
:103B1000089580910C0190910D01FC0131969C015A
:103B2000205E3F4F80E0919191118F5FE217F30784
:103B3000D1F70895E0910C01F0910D0180913C02C4
:103B40008083E0910C01F0910D01908180913B0206
:103B5000892B808380911A02882361F0E0910C0107
:103B6000F0910D019081892B80830E94891D811124
:103B700010921A0280910C0190910D010C94101278
:103B8000909347018093460108958295982F9C7CDD
:103B9000392F36953695282F237344E0249FC00192
:103BA0001124932F982B292F2A7A2695892F8575F2
:103BB000880F822B08950895CF93DF9300D000D013
:103BC0001F92CDB7DEB70F900F900F900F900F9010
:103BD000DF91CF910895089508950C94541383B7FD
:103BE000817F8C6083BF83B7816083BF7894889521
:103BF00083B78E7F83BF089508950895CF930E9461
:103C0000FC1D0E9442070E94FD1DC0E08C2F0E94F7
:103C10004508811104C0CF5FC032C1F701C081E007
:103C2000CF9108950E9433070C9490171F920F9222
:103C30000FB60F9211248F939F93AF93BF938091F0
:103C40003E0290913F02A0914002B0914102419604
:103C5000A11DB11D80933E0290933F02A0934002AC
:103C6000B0934102BF91AF919F918F910F900FBE82
:103C70000F901F90189582E084BD93E095BD9AEF58
:103C800097BD80936E0008952FB7F89480913E02FF
:103C900090913F02A0914002B09141022FBF089540
:103CA0002FB7F89460913E0270913F0280914002DC
:103CB000909141022FBF0895CF92DF92EF92FF9231
:103CC0000F931F932FB7F89440913E0250913F02FB
:103CD00060914002709141022FBF6A017B01EE2486
:103CE000FF248C0120E030E0C016D106E206F30686
:103CF00010F4415051099A01281B390BC9011F9139
:103D00000F91FF90EF90DF90CF9008951F920F9248
:103D10000FB60F9211248F939F93AF93BF9380910F
:103D20003E0290913F02A0914002B0914102019663
:103D3000A11DB11D80933E0290933F02A0934002CB
:103D4000B0934102BF91AF919F918F910F900FBEA1
:103D50000F901F9018950E944B0FF8942FEF87EA51
:103D600091E6215080409040E1F700C0000087E0DC
:103D700090EBDC018093600290936102A093620259
:103D8000B09363029CE088E10FB6F894A895809305
:103D900060000FBE90936000FFCF28E0929FF0017B
:103DA0001124E80FF11DE450FF4F9491892F8F707B
:103DB00092959F700895CF93C82FCB010E94CD1E7E
:103DC000282F30E080E1989FA0011124422B532B33
:103DD0004038510519F480E090E015C09770E92F44
:103DE000F0E088E0C89FE00DF11D112484E0EE0FA3
:103DF000FF1F8A95E1F7E20FF31FEE0FFF1FE05060
:103E0000F84985919491CF91089580E090E00895CC
:103E100008958091440280FF0BC06091110185E0FC
:103E2000689FB001112475956795759567952BC0AE
:103E300081FF09C06091110185E0689FB0011124E4
:103E40007595679520C082FF07C06091110185E0DC
:103E5000689FB001112417C0909145029923D1F0B9
:103E600060911001961788F72091110185E0289F35
:103E700090011124929FA001939F500D112470E096
:103E8000CA010E94E3266038710540F4611571058E
:103E900039F002C065E070E0862F08958FE708953D
:103EA00081E008958091440280FF08C060910F0175
:103EB00070E0759567957595679521C081FF06C07F
:103EC00060910F0170E07595679519C082FF04C07D
:103ED00060910F0170E010C0909145029923C1F0EC
:103EE00060910E019617A0F780910F01899FC00184
:103EF000112470E00E94E3266038710528F46115F2
:103F0000710521F0862F08958FE7089581E00895C7
:103F100061E070E0F4CF803F21F40E94091F819599
:103F200004C0813F29F40E94091F8093480208952C
:103F3000823F21F40E94091F819504C0833F29F428
:103F40000E94091F809347020895893F19F40E9437
:103F5000521F05C08A3F31F40E94521F8195809301
:103F6000490208958B3F21F40E94521F819504C09D
:103F70008C3F29F40E94521F80934A020895843F87
:103F800021F480914602816017C0853F21F4809121
:103F90004602826011C0863F21F48091460284600F
:103FA0000BC0873F21F480914602886005C0883F9E
:103FB00031F48091460280618093460208958D3FDE
:103FC00021F48091440281600BC08E3F21F48091E6
:103FD0004402826005C08F3F29F4809144028460CE
:103FE000809344020895803F39F48091480287FF0E
:103FF0006CC01092480269C0813F29F48091480248
:104000001816BCF362C090914702823F29F497FFD3
:104010005CC01092470259C0833F19F41916CCF3C3
:1040200054C0893F41F48091490218160CF04DC0EC
:10403000109249024AC08A3F29F48091490287FFC1
:1040400044C0F6CF8B3F39F480914A0287FF3DC0D0
:1040500010924A023AC08C3F29F480914A02181605
:10406000BCF333C0843F21F4809146028E7F17C099
:10407000853F21F4809146028D7F11C0863F21F457
:10408000809146028B7F0BC0873F21F480914602CE
:10409000877F05C0883F31F4809146028F7E8093F0
:1040A000460213C08D3F21F4809144028E7F0BC0E5
:1040B0008E3F21F4809144028D7F05C08F3F29F40B
:1040C000809144028B7F809344028091470281114A
:1040D0000EC08091480281110AC08091490281116D
:1040E00006C080914A02811102C0109245020895D3
:1040F00080913D0283FF7EC081ED95E00E944E06D7
:10410000809146021F928F938CEC95E09F938F9342
:104110000E94E7068AEC95E00E944E0680914702D5
:10412000282F082E000C330B3F938F9387EC95E0DC
:104130009F938F930E94E70685EC95E00E944E06C0
:1041400080914802282F082E000C330B3F938F9349
:1041500082EC95E09F938F930E94E70680EC95E0B8
:104160000E944E0680914902282F082E000C330B26
:104170003F938F938DEB95E09F938F930E94E7067B
:104180008BEB95E00E944E0680914A02282F082E64
:10419000000C330B3F938F9388EB95E09F938F93A5
:1041A0000E94E70685EB95E00E944E06809145024D
:1041B0001F928F9382EB95E09F938F930E94E70667
:1041C00080EB95E00E944E06809144021F928F93EF
:1041D0008DEA95E09F938F930E94E7068AEA95E027
:1041E0000E944E068DB79EB74C960FB6F8949EBFB0
:1041F0000FBE8DBF86E492E00E9459120E94441EB9
:10420000909343028093420208951F93CF93DF93CC
:1042100080914202909143020E945C1EAC019091F9
:104220004502992321F02091120130E006C020912F
:1042300013018AE0289F900111244217530708F4C4
:1042400085C080914702C0914802D09149021091E7
:104250004A02811107C0C11175C0D11173C011117B
:1042600071C074C09F3F19F09F5F9093450218166C
:1042700024F40E94091F809347028091470287FF20
:1042800005C00E94091F8195809347021C1624F4E3
:104290000E94091F809348028091480287FF05C051
:1042A0000E94091F8195809348026091470266230E
:1042B00031F1C0914802CC2311F1062E000C770B8E
:1042C000880B990B0E94DE2523E333E343E35FE38E
:1042D0000E9442260E94A625609347026C2FCC0FB5
:1042E000770B880B990B0E94DE2523E333E343E32E
:1042F0005FE30E9442260E94A625609348021D1695
:1043000024F40E94521F809349028091490287FF42
:1043100005C00E94521F819580934902111624F412
:104320000E94521F80934A0280914A0287FF05C073
:104330000E94521F819580934A02DF91CF911F9175
:104340000C9478209F3F09F08FCF97CFDF91CF91CA
:104350001F910895E6E4F2E085E0DF011D928A9561
:10436000E9F71092450210924402089584EF97E015
:104370000E944E061F9281E08F931F9285E08F93DB
:1043800086EA97E09F938F930E94E7060F900F9025
:104390000F900F900F900F9008958330E9F128F45B
:1043A000813061F0823009F10895853009F462C0EE
:1043B00008F449C0863009F474C00895809113014F
:1043C000262F30E0280F311D2F3F310524F4680FD0
:1043D0006093130103C08FEF809313018091130149
:1043E0001F928F938FED96E072C080911201262F5D
:1043F00030E0280F311D2F3F310524F4680F609302
:10440000120103C08FEF80931201809112011F925D
:104410008F938DEC96E05BC080911101262F30E0E8
:10442000280F311D2F3F310524F4680F60931101CF
:1044300003C08FEF80931101809111011F928F9320
:104440008AEB96E044C080911001262F30E0280FBF
:10445000311D2F3F310524F4680F6093100103C014
:104460008FEF80931001809110011F928F9385EA46
:1044700096E02DC080910F01262F30E0280F311DCE
:104480002F3F310524F4680F60930F0103C08FEFB5
:1044900080930F0180910F011F928F938CE896E01B
:1044A00016C080910E01262F30E0280F311D2F3FBE
:1044B000310524F4680F60930E0103C08FEF8093E1
:1044C0000E0180910E011F928F9381E796E09F93DA
:1044D0008F930E94E7060F900F900F900F90089512
:1044E000833081F128F4813059F08230D1F0089581
:1044F000853009F449C0B8F1863009F456C00895F2
:1045000080911301681720F4861B8093130102C069
:1045100010921301809113011F928F9382E696E00F
:1045200054C080911201681720F4861B80931201F9
:1045300002C010921201809112011F928F9380E5A8
:1045400096E043C080911101681720F4861B809388
:10455000110102C010921101809111011F928F93DD
:104560008DE396E032C080911001681720F4861B1D
:104570008093100102C010921001809110011F92CF
:104580008F9388E296E021C080910F01681720F494
:10459000861B80930F0102C010920F0180910F01C2
:1045A0001F928F938FE096E010C080910E016817E4
:1045B00020F4861B80930E0102C010920E018091A0
:1045C0000E011F928F9384EF95E09F938F930E942B
:1045D000E7060F900F900F900F900895CF93C82F7C
:1045E0001F928F9389EF98E09F938F930E94E70625
:1045F00081E090E0A0E0B0E0BC01CD0104C0660F16
:10460000771F881F991FCA95D2F70E94841B0F90AD
:104610000F900F900F90CF910C949017CF938732FB
:10462000A8F58E3108F02BC1803109F49FC0F8F451
:10463000873009F464C0A8F4863009F024C1809161
:104640003D02817F8E7F80933D028EEF98E00E9435
:104650004E068EEE9BE00E944E0681E080934C0257
:104660004CC08B30F1F18E3009F46CC00CC1863136
:1046700009F4B0C020F4813109F4EDC004C18931DE
:1046800009F491C08B3109F449C0FDC0883349F168
:1046900050F4893209F4F1C0853309F4EEC0873251
:1046A00009F0F1C0EAC0833409F4E7C028F48A3382
:1046B00008F4E9C08953E4C0883409F0E4C00E94DA
:1046C00090178DED9BE00E944E062FEF83ED90E357
:1046D000215080409040E1F700C000000E94AB1ED6
:1046E0000CC085E299E05CC084EC9BE00E944E0621
:1046F00080913D02816080933D02C1E0C9C08091FC
:104700003D02C82FC17080FFEFCF80ED9BE00E947B
:104710004E0680913D02817F8E7F3DC090913D028B
:1047200091FBCC27C0F981E0C827892FC0FB81F914
:1047300080933D02CC2319F087EB9BE027C089EAE8
:104740009BE02EC090913D0292FBCC27C0F981E006
:10475000C827892FC0FB82F980933D02CC2319F032
:104760008AE99BE013C08AE89BE01AC090913D0261
:1047700093FBCC27C0F981E0C827892FC0FB83F9C0
:1047800080933D02CC2351F08EE79BE00E944E06C1
:1047900080913D02816080933D027AC081E79BE079
:1047A0000E944E06AACF82E69BE00E944E068EE350
:1047B0009BE00E944E0688EF9AE00E944E068BEC2A
:1047C0009AE00E944E0681E89AE00E944E0683E538
:1047D0009AE0E6CF85E49AE00E944E060E94041219
:1047E0001F928F938BE29AE09F938F930E94E7062C
:1047F00080910A011F928F9384E19AE09F938F9397
:104800000E94E7068091B2011F928F9381E09AE0A7
:104810009F938F930E94E70680910B011F928F93C5
:104820008EEE99E09F938F930E94E7060E94501EA0
:104830009F938F937F936F9387ED99E09F938F93CF
:104840000E94E7068DB79EB746960FB6F8949EBFB6
:104850000FBE8DBF52CF0E949017C0910B0181E017
:10486000C827C0930B01CC2329F08DEC99E00E945E
:104870004E060EC082EC99E093CF80E001C08D51CE
:104880000E94EE223ACF80EC99E00E944E06C0E0F2
:104890008C2FCF91089580E0089580E00895CF9304
:1048A000C82F80914C02813079F020F0823009F4D9
:1048B0004DC044C1E0910C01F0910D018081815205
:1048C000823008F03DC108C0E0910C01F0910D016B
:1048D00080818152823060F48C2F0E944B248111A0
:1048E00004C08C2F0E940E232FC081E090E02CC0CA
:1048F0008C2F0E944D24811126C0C431E1F070F448
:10490000CB3081F0C031D1F40E94B62181EF98E024
:104910000E944E0682E080934C0215C0C93259F0C5
:10492000C83361F48EEF98E00E944E0685EF98E060
:104930000E944E0608C010924C0204C18FEE98E00F
:104940000E944E06FFC081E08170FEC0C43228F58F
:10495000CE3108F0C1C0CB30A1F1D0F4C73009F09E
:10496000D3C08EE18093130182E3809312018AE029
:104970008093110184E18093100188E080930F01FE
:1049800088E280930E0185E997E00E944E06BFC041
:10499000C33149F1C431C1F0B7C0CB3409F4A9C067
:1049A00028F4C93289F0C83361F0AEC0C13509F4CA
:1049B0009EC0C23509F499C0CE3409F0A5C06AE0A2
:1049C0009EC00E94B621A3C080914B02882319F09B
:1049D00010924B029CC082EA97E00E944E0681E052
:1049E00080934C02B1C08CE797E00E944E068AE6A5
:1049F00097E00E944E06809113011F928F9387E6E5
:104A000097E09F938F930E94E70685E697E00E94C8
:104A10004E0683E597E00E944E06809112011F9298
:104A20008F9380E597E09F938F930E94E7068EE433
:104A300097E00E944E068FE397E00E944E06809119
:104A400011011F928F938CE397E09F938F930E94A5
:104A5000E7068AE397E00E944E0689E297E00E940B
:104A60004E06809110011F928F9386E297E09F93EC
:104A70008F930E94E70684E297E00E944E068FE043
:104A800097E00E944E0680910F011F928F938CE059
:104A900097E09F938F930E94E7068AE097E00E9439
:104AA0004E0683EF96E00E944E0680910E011F9203
:104AB0008F9380EF96E09F938F930E94E7068EEE90
:104AC00096E00E944E068DB79EB748960FB6F894B2
:104AD0009EBF0FBE8DBF1BC0CE51EC2FF0E0E55C3A
:104AE000FE4F808180934B0212C061E003C061E001
:104AF00006C06AE080914B020E94CD2108C08091DF
:104B00004B020E94702203C083E997E013C080919A
:104B10004B02882369F01F928F938DE897E09F9353
:104B20008F930E94E7060F900F900F900F9004C094
:104B30008AE897E00E944E0681E006C010924C027F
:104B400080E002C080E000CFCF9108950E94AD25A3
:104B50006894B1110C943C2608950E94212688F097
:104B60009F5798F0B92F9927B751B0F0E1F0660F31
:104B7000771F881F991F1AF0BA95C9F714C0B13072
:104B800091F00E943B26B1E008950C943B26672FDC
:104B9000782F8827B85F39F0B93FCCF386957795A1
:104BA0006795B395D9F73EF490958095709561958A
:104BB0007F4F8F4F9F4F0895E89409C097FB3EF4B5
:104BC00090958095709561957F4F8F4F9F4F99235A
:104BD000A9F0F92F96E9BB279395F69587957795D8
:104BE0006795B795F111F8CFFAF4BB0F11F460FF98
:104BF0001BC06F5F7F4F8F4F9F4F16C0882311F0F0
:104C000096E911C0772321F09EE8872F762F05C003
:104C1000662371F096E8862F70E060E02AF09A959E
:104C2000660F771F881FDAF7880F9695879597F993
:104C3000089557FD9058440F551F59F05F3F71F08C
:104C40004795880F97FB991F61F09F3F79F08795F3
:104C50000895121613061406551FF2CF4695F1DF7C
:104C600008C0161617061806991FF1CF869571050C
:104C7000610508940895E894BB2766277727CB0140
:104C800097F908950E9455260C94C6260E94B826CE
:104C900038F00E94BF2620F0952311F00C94AF2627
:104CA0000C94B52611240C943C260E94192670F30E
:104CB000959FC1F3950F50E0551F629FF001729FC1
:104CC000BB27F00DB11D639FAA27F00DB11DAA1FD0
:104CD000649F6627B00DA11D661F829F2227B00D1D
:104CE000A11D621F739FB00DA11D621F839FA00DA8
:104CF000611D221F749F3327A00D611D231F849FF8
:104D0000600D211D822F762F6A2F11249F5750404E
:104D10009AF0F1F088234AF0EE0FFF1FBB1F661FC9
:104D2000771F881F91505040A9F79E3F510580F092
:104D30000C94AF260C943C265F3FE4F3983ED4F3EA
:104D4000869577956795B795F795E7959F5FC1F736
:104D5000FE2B880F911D9695879597F9089597F9E1
:104D60009F6780E870E060E008959FEF80EC089511
:104D700000240A941616170618060906089500243A
:104D80000A9412161306140605060895092E0394B4
:104D9000000C11F4882352F0BB0F40F4BF2B11F428
:104DA00060FF04C06F5F7F4F8F4F9F4F0895991B27
:104DB00079E004C0991F961708F0961B881F7A9512
:104DC000C9F78095089597FB072E16F4009407D035
:104DD00077FD09D00E94FD2607FC05D03EF4909592
:104DE00081959F4F0895709561957F4F0895EE0FBF
:104DF000FF1F0590F491E02D0994AA1BBB1B51E104
:104E000007C0AA1FBB1FA617B70710F0A61BB70B3A
:104E1000881F991F5A95A9F780959095BC01CD01DF
:104E20000895A0E0B0E0E7E1F7E20C94B529AE0107
:104E30004B5F5F4FFA0161917191AF0180915C020C
:104E400090915D020E942727E2E00C94D129ACE00A
:104E5000B0E0EDE2F7E20C94A5297C016B018A0138
:104E6000FC0117821682838181FFBDC1CE010196AC
:104E70004C01F7019381F60193FD859193FF819198
:104E80006F01882309F4ABC1853239F493FD859114
:104E900093FF81916F01853229F4B70190E00E9460
:104EA0000F29E7CF512C312C20E02032A0F48B3297
:104EB00069F030F4803259F0833269F420612CC0FB
:104EC0008D3239F0803339F4216026C022602460AD
:104ED00023C0286021C027FD27C030ED380F3A30AD
:104EE00078F426FF06C0FAE05F9E300D1124532EA1
:104EF00013C08AE0389E300D1124332E20620CC07E
:104F00008E3221F426FD6BC1206406C08C3611F46C
:104F1000206802C0883641F4F60193FD859193FF25
:104F200081916F018111C1CF982F9F7D955493304E
:104F300028F40C5F1F4FFFE3F9830DC0833631F077
:104F4000833771F0833509F05BC022C0F80180819E
:104F500089830E5F1F4F44244394512C540115C084
:104F60003801F2E06F0E711CF801A080B18026FFBD
:104F700003C0652D70E002C06FEF7FEFC5012C8785
:104F80000E9404292C0183012C852F77222E17C023
:104F90003801F2E06F0E711CF801A080B18026FF8D
:104FA00003C0652D70E002C06FEF7FEFC5012C8755
:104FB0000E94F9282C012C852068222E830123FCD5
:104FC0001BC0832D90E048165906B0F4B70180E26B
:104FD00090E00E940F293A94F4CFF50127FC8591C7
:104FE00027FE81915F01B70190E00E940F293110E7
:104FF0003A94F1E04F1A51084114510471F7E5C099
:10500000843611F0893639F5F80127FF07C0608131
:105010007181828193810C5F1F4F08C06081718113
:10502000072E000C880B990B0E5F1F4F2F76722EE8
:1050300097FF09C090958095709561957F4F8F4F30
:105040009F4F2068722E2AE030E0A4010E94472979
:10505000A82EA81844C0853729F42F7EB22E2AE046
:1050600030E025C0F22FF97FBF2E8F36C1F018F443
:10507000883579F0B4C0803719F0883721F0AFC097
:105080002F2F2061B22EB4FE0DC08B2D8460B82E60
:1050900009C024FF0AC09F2F9660B92E06C028E0E1
:1050A00030E005C020E130E002C020E132E0F8014C
:1050B000B7FE07C060817181828193810C5F1F4FB1
:1050C00006C06081718180E090E00E5F1F4FA401F7
:1050D0000E944729A82EA818FB2DFF777F2E76FE69
:1050E0000BC0372D3E7FA51450F474FE0AC072FC2D
:1050F00008C0372D3E7E05C0BA2C372D03C0BA2C10
:1051000001C0B52C34FF0DC0FE01EA0DF11D8081F8
:10511000803311F4397E09C032FF06C0B394B394D2
:1051200004C0832F867809F0B39433FD13C030FF99
:1051300006C05A2CB31418F4530C5B18B32CB314D8
:1051400068F4B70180E290E03C870E940F29B39495
:105150003C85F5CFB31410F43B1801C0312C34FF5B
:1051600012C0B70180E390E03C870E940F293C8584
:1051700032FF17C031FD03C088E790E002C088E528
:1051800090E0B7010CC0832F867859F031FF02C040
:105190008BE201C080E237FD8DE2B70190E00E9412
:1051A0000F29A51438F4B70180E390E00E940F297D
:1051B0005A94F7CFAA94F401EA0DF11D8081B7014A
:1051C00090E00E940F29A110F5CF332009F451CEB1
:1051D000B70180E290E00E940F293A94F6CFF701E0
:1051E0008681978102C08FEF9FEF2C96E2E10C94AD
:1051F000C129FC010590615070400110D8F78095DD
:1052000090958E0F9F1F0895FC0161507040019092
:105210000110D8F7809590958E0F9F1F08950F93DA
:105220001F93CF93DF93FB01238121FD03C08FEFF9
:105230009FEF28C022FF16C0468157812481358107
:105240004217530744F4A081B1819D012F5F3F4F66
:10525000318320838C93268137812F5F3F4F3783A3
:10526000268310C0EB01092F182F0084F185E02D53
:105270000995892BE1F68E819F8101969F838E830C
:10528000812F902FDF91CF911F910F910895FA01F7
:10529000AA27283051F1203181F1E8946F936E7F75
:1052A0006E5F7F4F8F4F9F4FAF4FB1E03ED0B4E066
:1052B0003CD0670F781F891F9A1FA11D680F791FA7
:1052C0008A1F911DA11D6A0F711D811D911DA11DB8
:1052D00020D009F468943F912AE0269F11243019C8
:1052E000305D3193DEF6CF010895462F4770405D63
:1052F0004193B3E00FD0C9F7F6CF462F4F70405D12
:105300004A3318F0495D31FD4052419302D0A9F76C
:10531000EACFB4E0A6959795879577956795BA9566
:10532000C9F700976105710508959B01AC010A2E2C
:1053300006945795479537952795BA95C9F7620F03
:10534000731F841F951FA01D08952F923F924F92A7
:105350005F926F927F928F929F92AF92BF92CF9205
:10536000DF92EF92FF920F931F93CF93DF93CDB70E
:10537000DEB7CA1BDB0B0FB6F894DEBF0FBECDBF86
:1053800009942A88398848885F846E847D848C8457
:105390009B84AA84B984C884DF80EE80FD800C8160
:1053A0001B81AA81B981CE0FD11D0FB6F894DEBF43
:0C53B0000FBECDBFED010895F894FFCFB3
:1053BC00670A580B350B010BCD0A01011B0228089B
:1053CC00140A321E4F4B004E4700424154202573A5
:1053DC000A00404D3622390905BC04860464042BAE
:1053EC00049E03B703D003E9030904010203040577
:0653FC000607080900008D
:106800008800EA44E944E244040005000600070069
:10681000080009000A000B000C000D000E000F001C
:1068200010001100120013001400150016001700CC
:10683000180019001A001B001C001D001E001F007C
:10684000200021002200230024002500260027002C
:10685000280029002A002B002C002D002E002F00DC
:1068600030003100000033003400350036003700BE
:10687000380039003A003B003C003D003E003F003C
:1068800040004100420043004400450046004700EC
:10689000480049004A004B004C004D004E004F009C
:1068A000500051005200530054005500560057004C
:1068B000580059005A005B005C005D005E005F00FC
:1068C00060006100620063006400F1A18500670060
:1068D000680069006A006B006C006D006E006F005C
:1068E0007000710072007300890087008A008B00BD
:1068F000E000E100E200E300E400E500E600E7007C
:106900000100010001000100EA4401000100E2442D
:106910000100010001000100460001004A004B0097
:10692000010001004700480001000100E9440100A6
:106930000100010001000100010001003A003B00DC
:106940003C003D003E003F0040004100420043004B
:10695000010035004C0039000100440045005200A0
:1069600049000100010050004F0029004D004E0079
:1069700051000100010001000100010001000100BF
:1069800001000100010001000100010001000100FF
:1069900001000100010001000100010001004D00A3
:1069A0004A004E004B0001000100010001000100FF
:1069B00001000100010001000100010001000100CF
:1069C00001000100010001000100010001000100BF
:1069D00001000100010001000100010001000100AF
:1069E0000100010001000100490001000100010057
:1069F000010001000100010001000100010001008F
:00000001FF
